:020000040000FA
:06000000ACEF01F012005C
:020006001200E6
:06000800A0EF00F0120061
:02000E000100EF
:0C001000940300008A00000007000000BC
:04001C00720ED36E1F
:10002000C26A0D0EC16EC06A430E926E010E936ECF
:10003000C50E946E89688A68FD0E8B6E0D0EE66E95
:10004000040EE66ED90EE66E12EC01F0E552E552B2
:10005000E552870EE66E6FEC01F0E552C8EC01F058
:10006000C3EC01F0000901E0FBD7BAEC01F0F3CFDB
:1000700010F0F4CF11F0560E0D6E010E0E6E10C082
:1000800008F011C009F049EC01F008C010F009C0F7
:1000900011F010C091F08F0EE66E6FEC01F0E5529A
:1000A000C8EC01F0C3EC01F0000901E0FBD7BAECA9
:1000B00001F0F3CF10F0F4CF11F0560E0D6E010EDB
:1000C0000E6E10C008F011C009F049EC01F008C034
:1000D00010F009C011F0030E1102F3CF11F010025D
:1000E000F3CF10F0F4501126105000019127020EAA
:1000F000E76E9119E8AE02D0E73402D0E750915D87
:100100000BE3060EE76E9119E8AE02D0913503D0ED
:10011000E750D880915502E2020E916F91C0E9FF3D
:10012000EA6AE9BEEA688A0EE926000EEA22EFCF03
:1001300092F0F288F18CD09EF28CF28EFFD71200F2
:10014000DACFE4FFE2CFDAFFE9CFE4FFEACFE4FF62
:10015000E652F2A210D0F292000192070CE18B76E7
:1001600091C0E9FFEA6AE9BEEA688A0EE926000E54
:10017000EA22EFCF92F0E552E5CFEAFFE5CFE9FFC3
:06018000E5CFDAFF1100DB
:0A0186000E0EF66E000EF76E000E6E
:10019000F86E00010900F550856F0900F550866F73
:1001A00003E1856701D03DD00900F550806F09005B
:1001B000F550816F0900F550826F09000900F55074
:1001C000E96E0900F550EA6E090009000900F550D2
:1001D000836F0900F550846F09000900F6CF87F09E
:1001E000F7CF88F0F8CF89F080C0F6FF81C0F7FF25
:1001F00082C0F8FF0001835302E1845307E0090045
:10020000F550EE6E8307F8E28407F9D787C0F6FF52
:1002100088C0F7FF89C0F8FF00018507000E865BE4
:04022000BFD7120032
:0C022400D9CFE6FFDACFE6FFE1CFD9FF2B
:10023000E2CFDAFFC26AC06AFC0EDB407F0B3C0BE8
:10024000C26EFC0EDB38F00B300B106EFB0EDB5079
:100250000F0B1010C16EFD0EDB50040DF350380B68
:10026000116EFD0EDB380F0B070B106EFD0EDB5011
:10027000800B10101110C06EFC0EDBAE03D09E9CE4
:100280009D8CF28CC280E552E5CFDAFFE7CFD9FF33
:0202900012005A
:0E029200006A0EAE52EF01F00D6C0E1EE86A0F
:1002A0000E22001E09AE5AEF01F0086C091EE86A22
:1002B0000922001E86EC01F009BE6AEF01F000AED3
:1002C000000C086C091EE86A0922046C051EE86A25
:0E02D0000522000C00BE61EF01F00188FF0C5A
:0202DE00D9CF76
:1002E000E6FFDACFE6FFE1CFD9FFE2CFDAFFC30EB8
:1002F000C214106EFD0EDB407F0B3C0B1010C26E63
:0C030000E552E5CFDAFFE7CFD9FF12008D
:04030C00056A046A10
:10031000100EE76ED89008360936043605360D50B3
:10032000045C0E50055805E30D50045E0E50055A4E
:08033000082AE72EF0D71200A5
:08033800000EF36E00EE00F070
:10034000030E01D81200EA6002D0EE6AFCD7F35027
:08035000E9601200EE6AFCD71F
:0803580012EE00F022EE00F0AD
:10036000F86A019CC3EC00F003EC00F00EEC00F026
:04037000FBD71200A5
:0C037400C450136E126AC3501210F36ED6
:0603800013C0F4FF12009F
:0A038600C250020B01E0010E12004C
:04039000C282120013
:070394000101010204080A47
:020000040030CA
:0100010008F6
:0100020019E4
:010003001EDE
:0100050000FA
:010006008079
:010008000FE8
:01000900C036
:01000A000FE6
:01000B00E014
:01000C000FE4
:01000D0040B2
:00000001FF
